:020000020000FC
:0200000022C01C
:0400140089C0CCC013
:02001A00CEC056
:100020000FC10D0A626B2373626C2D666C6F6823BF
:100030003838765F70706D32306B5F7430322831D3
:10004000356730290D0A04E00EBF0FEF0DBF03E83E
:1000500005B900E804B908E208B90AE307B905E1FF
:100060000BB90AEB0AB901E000937E0001E00093AE
:100070007F0002E005BD02E000938100772788271A
:100080009927B1E0A0E000271DE20D931A95E9F74A
:100090000DD304E6902E19B11570153069F01430A7
:1000A00041F0113019F001E011E008C00CE01AE055
:1000B00005C008E114E102C002E318E20093210147
:1000C00010932201589859983ED13DD110D12FD18B
:1000D00011D12DD112D12BD106EF302E00E0D02E30
:1000E00001E005BB00936E0003E206BB00936F00C6
:1000F00002EE00937C0059D178942AE083FFFECF72
:100100000091190110911A01877F0C541440A8F72F
:100110002A95A1F7F894F4D0F3D0F2D078940EE1B8
:1001200000932401B1D117C32FB64091860050919E
:1001300087006091810066FF1AC06F7B6093810029
:10014000742E852E9F7760911701461B60911801D0
:10015000560B483A61E6560730F4483863E15607D3
:1001600010F0906823C0992009F19A941FC0606430
:100170006093810083FD1AC04093170150931801CA
:1001800097FF14C09F77471958094093190150935E
:100190001A01483968E0560730F7403263E05607E5
:1001A00010F38860492D443609F093942FBE1895BA
:1001B0002FB67E7F2FBE18952FB67068EE2009F0FF
:1001C000EA94992009F09A9440912B01442319F55F
:1001D00040912901442329F05D984A9540932901D3
:1001E00016C040912A01442329F05F984A95409314
:1001F0002A010DC040912701409329014091280117
:1002000040932A014AE140932B01806817C048E0DF
:1002100040932B0113C04A9540932B0187FF0BC0DD
:10022000463139F0433129F0463019F0433019F4A2
:100230008F772F9801C02F9A5D9A5F9A2FBE1895DD
:100240002FB676FD32C0906140B745FD9F7E432DAD
:10025000552D541738F44A9469F450912101452ED4
:100260004A9507C039F04A9429F450912201452E4D
:100270004395342E706475FF03C081FF5B9807C0FF
:1002800074FF03C081FF419802C081FF4498432D51
:10029000425A3AF44A5F433040F047704A95F1F7CA
:1002A00004C04095459546BD1EC075FF03C080FF44
:1002B0005B9A07C074FF03C080FF419A02C080FFB1
:1002C000449A432D4F93459546BD4F917F7B4D39C1
:1002D00018F482608E7F07C0463F18F08D7F8160E2
:1002E00002C08D7F8E7F93FD81602FBE189538EC04
:1002F00010E509C034EB14E606C030EA18E703C085
:1003000034E618EC00C0002706BD4598419A06B5B2
:100310000032E9F7459A419828E0002706BD06B566
:100320000317E9F72A95C9F71A9569F708951FE0A9
:1003300028E0002706BD06B50F3FE9F72A95C9F763
:100340001A95B1F7089510E828E0002706BD06B514
:100350000F3FE9F72A95C9F71A95B1F7089505E80F
:1003600000937A0000917B000F7B00937B0020912B
:100370007C0002EE00937C000000000005EC00937E
:100380007A00000000917A0006FDFCCF0091790010
:100390000F9305E000937A0000917B0000640093C6
:1003A0007B000F9120937C000895D9DF00932301F7
:1003B0009F7B073D48F40A3C50F40C3B58F40F3A3D
:1003C00060F400E014E00BC004E010E008C003E0BB
:1003D00011E005C002E012E002C001E013E000936A
:1003E00027011093280108958F7E83FF15C0009187
:1003F000190110911A01877F0C54144010F4002742
:100400001127169507951695079516950795202F90
:10041000045608F024E6F22F08958F7B20910C01FA
:1004200010910B0100910A01011B00930A01009138
:100430000B01020B00930B0100910C010040009393
:100440000C012091090110910801009107012695E6
:1004500017950795269517950795209309012093E1
:1004600008012093070120910A01200F20930A011F
:1004700020910B01211F20930B0100E020910C0122
:10048000201F20930C010895C0E8DBEBC0931101FD
:10049000D09312012FEF3FE120930D0130930E0115
:1004A00020930F0130931001E1E0E09306013FEF4C
:1004B000309305012FEF209304010895F894000074
:1004C00000918400109185000093000110930101B8
:1004D0000C0F1D1F109389000093880071607894A1
:1004E0000091040110910501E091060100931301B0
:1004F00010931401EE2329F03FEF30931301309352
:100500001401E69517950795E6951795079520919F
:10051000040130910501E0910601201B310BE04000
:100520000091000110910101C0910201D0910301DD
:1005300000930201109303010C1B1D0B0093150186
:1005400010931601200F311F10E0E11FEE2351F42C
:10055000332341F4213E30F431E02CE4FF2011F448
:100560000FEFF02E2093040130930501E093060174
:10057000E23008F099DF00910701020F00930701B4
:1005800000910801031F00930801009109010E1F4B
:1005900000930901E69537952795E69537952795B8
:1005A000E69537952795E6953795279520930D0184
:1005B00030930E01FF2001F420930F0130931001BE
:1005C0000895C0910D01D0910E0178DF089570FD5E
:1005D000FECFD0911401C0911301F8940000009156
:1005E0008400109185000C0F1D1F1093890000934B
:1005F0008800716078940895C0910F01D091100126
:10060000F894000000918400109185000C0F1D1FCC
:1006100010938900009388007160789484FDE4DE73
:1006200085FD18D086FDF9DE96FDBFDE70FDFECF9C
:100630000895C0911101D091120140DF0091000195
:100640000F70D01BDC3808F4DBEBD093120141D0E3
:1006500040D008958F7D0F2F0D1908F409E01091F7
:100660000601112321F410910501103438F0916036
:10067000926019E1011760F0012F0AC0103238F0C2
:100680009E7F926012E3011718F0012F01C09C7F3A
:1006900095FF09C02EE1021710F40EE104C028E214
:1006A000021708F0022F0095502E0895F9E006EF8A
:1006B000302E502E08E208B905E10BB90091210156
:1006C000402E8160977F9062089504E00A95F1F7CB
:1006D000089576FDFECF76FFFECF089508952F93FF
:1006E0003F93797F71FD02C060DEFCCF797F71FDA1
:1006F00002C05BDEFCCF00911F01109120013F91F1
:100700002F910895ECDF202F312FE9DF021B130B0F
:1007100010F4109500951123A9F7007F002391F79D
:1007200020931B0130931C0136952795369527950C
:1007300000E014E63327EE273395332309F4E395DD
:10074000021B3F933327130B3F91B0F730931D01EA
:10075000E0931E010895AADFC1DF46DE26DEFA30EF
:10076000E0F30EE10095502E332703E805B905E1CB
:100770000BB90BE10A95F1F73BD141D19B7F00E02A
:100780000093250108E2E02E7FDE53DF94FF10C0C6
:1007900070FD02C0946013C09CDF94FDF9CF00E0AF
:1007A00000932501EFD0F5D008D11EDE42DF31C025
:1007B00070FD02C0946003C08CDF94FFF9CFE2D0DB
:1007C00038DF94FD08C070FD02C094600BC081DF6B
:1007D00094FFF9CF07C070FD02C0946003C079DFB9
:1007E00094FDF9CFD6D000DE24DF94FF08C070FD61
:1007F00002C094600BC06DDF94FDF9CF07C070FD9F
:1008000002C0946003C065DF94FFF9CFD6D022DF29
:1008100010DF94FD08C070FD02C094600BC059DF6A
:1008200094FFF9CF07C070FD02C0946003C051DF90
:1008300094FDF9CFC9D0B9DDFCDE94FF08C070FD8E
:1008400002C094600BC045DF94FDF9CF07C070FD76
:1008500002C0946003C03DDF94FFF9CFC9D0E9DE48
:1008600094FD08C070FD02C094600BC032DF94FF9D
:10087000F9CF07C070FD02C0946003C02ADF94FD69
:10088000F9CFBDD0032D063F09F465CF992021F49F
:1008900062CFEE2009F45FCF00910601002321F41E
:1008A00000910501003250F00091250192FD0027D2
:1008B0000395009325019B7F0C3338F00FEFF02E4A
:1008C00080DE87DE9F7D7B7F02C0B3DE5FCF50D0AE
:1008D00070FF32C0806490DE55D073DE78DE3ED08B
:1008E00070FF2AC0806188DE54D06BDE70DE40D09D
:1008F00070FF22C0806280DE60D063DE68DE2ED0B2
:1009000070FF1AC0906478DE5FD05BDE60DE30D0AE
:1009100070FF12C071DE6CD054DE59DE1FD070FF44
:100920000BC06ADE6CD04DDE52DE992009F413CF85
:1009300000910601002319F09062977F0ECF977FF8
:10094000FF2041F0FA9429F00F2D013011F0023010
:1009500009F49860BCCFF894A9DE75CB70FF0895B8
:1009600000B705FFFBCFB1DE00B705FFF7CF089555
:1009700070FF089500B705FDFBCFA7DE00B705FDAA
:10098000F7CF0895459A80FF439807EE00937C00C7
:10099000089500E000936E0000007F7E7F7D81FD62
:1009A00002C076FD03C05B9880FF449A01E000938B
:1009B0006E0006EE00937C000895439A80FF5C98D9
:1009C00000EE00937C00089500E000936E000000AC
:1009D00070617F7D81FD02C076FD03C0449880FF79
:1009E000419A01E000936E0007EE00937C000895A9
:1009F0005C9A80FF459806EE00937C00089500E025
:100A000000936E0000007F7E706281FD02C076FD63
:100A100003C0419880FF5B9A01E000936E0000EEF6
:060A200000937C00089524
:00000001FF
